:1000000019C033C032C031C030C02FC02EC02DC087
:100010002CC02BC02BC160C028C050C026C025C03A
:1000200024C023C022C021C020C01FC01EC01DC0CC
:100030001CC01BC011241FBECFEFD2E0DEBFCDBF5E
:1000400011E0A0E0B1E0ECEBF5E002C005900D920C
:10005000A830B107D9F711E0A8E0B1E001C01D92C6
:10006000AF31B107E1F702D0A7C2CACFEF92FF923A
:100070000F931F93CF93DF93A8D04DD084E690E0E9
:100080003CD081E5E82E8FD085359105E1F78BD006
:10009000182F89D0F82E87D0082F85D0982F1430AC
:1000A00091F78F2D80278E25891769F7DF2DC0E006
:1000B000802F90E08C2B9D2B20D0E5CF1F920F92AC
:1000C0000FB60F9211245A985C985F982B9A0F9054
:1000D0000FBE0F901F9018951F920F920FB60F92A0
:1000E00011248F938BB1877D8BB92B985F9A8F9159
:1000F0000F900FBE0F901F90189578948FEF91E09E
:1001000090930E0180930D0108952091110130917B
:100110001201C90108951BB815B88AB188628AB95D
:10012000239A8AB184698AB982E08093800089E148
:1001300080938100EFE6F0E08081836080838FEF21
:1001400091E090938700809386001092890010922E
:1001500088008FE080937E0083E080937F00EAE751
:10016000F0E080818F77808380E480937B00089526
:10017000FC01519A88E08093C100662359F0809178
:10018000C00085FFFCCF80818093C600615011F0D4
:100190003196F5CF8091C00085FFFCCF519880E16A
:1001A0008093C10008958091C00087FFFCCF8091AB
:1001B000C60090E00895982F8091C00085FFFCCF85
:1001C0009093C60080E090E0089588E08093C4009A
:1001D0001092C00086E88093C20088E18093C1003D
:1001E0008AB183608AB9519A8BED90E063ED70E03B
:1001F00072D008952098289AEFE6F0E0808180621E
:100200008083E1E8F0E08081826C80830895209112
:1002100001018091130190911401892B79F4B09B15
:10022000F8CF81E086BB109214011092130184E193
:10023000809301012FEF3FEFC90108954091130111
:10024000509114011092140110921301CA01855F9C
:1002500091408F5C974040F4222311F02150C9F661
:10026000109201019A01E8CF2AE0D3CF1F920F929A
:100270000FB60F9211242F933F934F938F939F9319
:100280002091860030918700220F331F409181001A
:1002900046FD1CC080910A0190910B01281B390B6F
:1002A0003093140120931301109285001092840062
:1002B00080E44827409381009F918F914F913F9117
:1002C0002F910F900FBE0F901F90189530930B0138
:1002D00020930A01EDCF0F931F93CF93DF938C01EF
:1002E000EB01009731F46115710519F420E030E05D
:1002F00037C081E090E06EE070E038D0FC019C01F6
:10030000009771F180E88383209771F0D387C287CB
:1003100081E883838091150190911601892B21F446
:10032000F0931601E093150101151105C9F011872D
:1003300000878381826083838091170190911801E7
:10034000892B71F4F0931801E09317018091190142
:1003500090911A01892B21F4F0931A01E09319016D
:10036000C901DF91CF911F910F9108950F931F93B2
:10037000CF93DF93689F8001699F100D789F100DC8
:100380001124C8010DD0EC01009721F060E070E06D
:10039000A8010BD1CE01DF91CF911F910F9108954C
:1003A000CF93DF93BC018230910510F462E070E0DE
:1003B000A0911D01B0911E01ED01E0E0F0E040E0F0
:1003C00050E021C0888199818617970769F48A8156
:1003D0009B81309719F09383828304C090931E0110
:1003E00080931D01FE0134C06817790738F4411568
:1003F000510519F08417950708F4AC01FE018A81B4
:100400009B819C01E9012097E9F641155105A9F16D
:10041000CA01861B970B049708F4BA01E0E0F0E0EC
:100420002AC08D919C91119784179507F9F4641750
:10043000750781F412968D919C911397309719F05E
:100440009383828304C090931E0180931D01FD015C
:1004500032964FC0CA01861B970BFD01E80FF91FAA
:100460006193719302978D939C9343C0FD018281A8
:1004700093819C01D9011097A1F680911B01909165
:100480001C01892B41F48091040190910501909306
:100490001C0180931B0140910601509107014115F9
:1004A000510541F44DB75EB780910201909103016F
:1004B000481B590B20911B0130911C012417350753
:1004C000B0F4CA01821B930B8617970780F0AB012B
:1004D0004E5F5F4F8417950750F0420F531F5093A4
:1004E0001C0140931B01F9016193719302C0E0E08C
:1004F000F0E0CF01DF91CF910895CF93DF93009784
:1005000009F450C0EC0122971B821A82A0911D01B0
:10051000B0911E01109709F140E050E0AC17BD0703
:1005200008F1BB83AA83FE0121913191E20FF31FF1
:10053000AE17BF0779F48D919C911197280F391F41
:100540002E5F3F4F3983288312968D919C9113978C
:100550009B838A834115510571F4D0931E01C0938A
:100560001D0120C012968D919C911397AD010097AB
:1005700011F0DC01D3CFFA01D383C28321913191F1
:10058000E20FF31FCE17DF0769F488819981280FE6
:10059000391F2E5F3F4FFA01318320838A819B816F
:1005A00093838283DF91CF910895DC0101C06D9325
:0C05B00041505040E0F70895F894FFCF50
:0805BC00FF3220001F010000C6
:00000001FF
